:020000040000FA
:020000003E2898
:08000800F000030EF1000A08EC
:10001000F20083010F3087058C10B90A39080339C3
:100020008A01820719281D2821283508860007160D
:1000300024283608860087162428370886000717E4
:10004000242838088600871772088A00710E8300FA
:10005000F00E700E09000F398A018207DB348234FA
:10006000E934E334B23473347B348334FB34F33413
:10007000BA3479345834B934203400348A018B01CD
:1000800083016400FF308500003086000F30870058
:100090008316E7308100FF3085000030860008308D
:1000A00087008312830140309F0083168C309F00AD
:1000B0008312103090009701831631309200831222
:1000C00004309200C001B901C101C201B501B601FD
:1000D000B701B801CE011E30CD0052264B08CC002E
:1000E0005308C3008C018D01831602308C008D01F2
:1000F0008312C0308B00D2268301871987284730AE
:10010000C200C1174110C11008308A0014286400D1
:100110008301CE0A00308A004308033982079328FE
:10012000E32800292D294608AA004508A90044080B
:10013000A800992500308A00430E03398207A328BE
:10014000C128CF28A3283408031DB3283308031D72
:10015000B3283208031DB328FF30B2003108031D55
:10016000B328FF30B10032082B20B50031082B2016
:10017000B60030082B200438B7002F082B20B80019
:10018000E22833082B200438B50032082B20B600B3
:1001900031082B20B70030082B20B800E2280A30A5
:1001A00034020318D62834080F39031D2B20B5005C
:1001B00033082B200438B60032082B20B700310852
:1001C0002B20B8003F294708AA00A901A8019925BA
:1001D000B50131080F39031D2B20B60030082B2044
:0C01E000B70037152F082B20B8003F296E
:10020000B501B5153516B601B701B80101308A0040
:100210004808073982071929182917291629152985
:1002200014291329B814B815B714B715B614B61590
:10023000B51401308A004908073982072C292B2977
:100240002A292929282927292629B8173816B7172E
:100250003716B6173616B5173F29B501B601B701DF
:10026000CE1D35290430B8003629B8014B080319D2
:100270003E284C0803193E29F030C3053F29F224DB
:100280000C2529257525AC2400245424E624362683
:040290000F26872886
:1008000083019F121F129F119F131F171F14AA010C
:10081000A9012A30A500A530A60097262A30A500F8
:10082000A730A60097261F1504308A004A0803390E
:100830008207282C242C202C2A30840003107126B7
:100840002A308400031071262A3084000310712698
:10085000290803192E2CA901FF30AA002A084802F2
:10086000031C352C2A08C800372C2A03C800480866
:10087000343C03183D2C3430C8004808043EC800FE
:10088000C80CC80C480C0739C8001F19452C831622
:100890002508A7002408A6001E08A50083011E083D
:1008A0008316A4008301080083019F121F129F1565
:1008B0009F131F171F14AA01A9012A30A500A930F0
:1008C000A60097262A30A500AB30A60097261F1554
:1008D00004308A004A08033982077C2C782C742C57
:1008E0002A308400031071262A30840003107126F8
:1008F0002A308400031071262A30840003107126E8
:1009000029080319862CA901FF30AA002A084902E8
:10091000031C8D2C2A08C9008F2C2A03C900490802
:10092000343C0318952C3430C9004908043EC900F2
:10093000C90CC90C490C0739C9001F199D2C831615
:100940002908AB002808AA001E08A90083011E0878
:100950008316A8008301080083019F161F129F11B0
:100960009F131F171F140430AA00A9012A30A500E5
:10097000A130A60097262A30A500A330A60097260E
:100980001F152A308400031071262A3084000310BA
:1009900071262A30840003107126A9012A08470213
:1009A000031CD52C2A08C700D72C2A03C7001F19FF
:1009B000D72C83162108A3002008A2001E08A1003E
:1009C00083011E088316A00083010800CD0BF12CC3
:1009D0000A30CD00CC080319F12CCC0BF12C4314B8
:1009E000C314080007110714BA0181010B1110107C
:1009F000FF308F008E0096019501083097000C1192
:100A00001014000000000000A3309600DC309500B8
:100A10000C110930970008000B08A3002319BA0A2B
:100A200023190B110C1D0C2D10100B08A3002319FA
:100A3000BA0A23190B110108BB00A000BC01071062
:100A40000714BC03000001082002031D282D1F2DE0
:100A500008003C08AA003B08A9003A08A800A70122
:100A60003F08AE003E08AD003D08AC00AB012A30A7
:100A7000A5002E30A6007E260319412D0318432D14
:100A80004E2D0000582D0130AE00AD01AC01AB0180
:100A90002A30A5002E30A600B726582D0130AE0012
:100AA000AD01AC01AB012A30A5002E30A6009B267B
:100AB0002A08BF002908BE002808BD000430AE0087
:100AC000AD01AC01AB012A30A5002E30A6009B265B
:100AD0002A308400031073262A3084000310732602
:100AE0002A3084000310732608002A30A5005230F3
:100AF000A6009B26A81F8C2DAE01AD01AC012E30A7
:100B0000A5002A30A600B7262E08AA002D08A900A5
:100B10002C08A8002B08A7002A0846020319922DCA
:100B20004B08CC002808C4002908C5002A08C600C4
:100B30000800A701A030AE008630AD000130AC0047
:100B4000AB01FF30A300A30A2A30A5002E30A60077
:100B5000B7260318A32D2A30A5002E30A6009B2609
:100B60002308B4001030AE002730AD00AC01AB015B
:100B7000FF30A300A30A2A30A5002E30A600B72616
:100B80000318BA2D2A30A5002E30A6009B26230874
:100B9000B300E830AE000330AD00AC01AB01FF3074
:100BA000A300A30A2A30A5002E30A600B7260318FA
:100BB000D12D2A30A5002E30A6009B262308B20096
:100BC0006430AE00AD01AC01AB01FF30A300A30A5D
:100BD0002A30A5002E30A600B7260318E72D2A30AC
:100BE000A5002E30A6009B262308B1000A30AE00D7
:100BF000AD01AC01AB01FF30A300A30A2A30A50070
:100C00002E30A600B7260318FD2D2A30A5002E3061
:100C1000A6009B262308B0002A08AF000800C11CCC
:100C2000252EC110411043080339031D292E430E00
:100C3000A000200A0339A000033C0319A001430EC1
:100C4000F0392004C300C30E352E411C352EC110CF
:100C500041104B08CC00430A0339A000033C0319A0
:100C6000A0014308F0392004C30008008719452E6D
:100C700042080311103C031DC20A420803110F3C35
:100C80000319C1140319C117512E42080314013C62
:100C900003184F2EC11B4F2E4114C117512EC201F4
:100CA000C1130800830100306726D0000130672699
:100CB000D10002306726D20003306726CA00043014
:100CC0006726D30005306726CB0083010800830127
:100CD00003178D0083168C010C1483120C088301FA
:100CE000080084037A2E840384038403800C840A1E
:100CF000800C840A800C840A800C0800A503A503DC
:100D0000A503A603A603A6030430A20003108A2E9F
:100D1000A50AA60A260884000008A1002508840068
:100D200021080002031D962EA20B882E0800023017
:100D3000A20003109E2E0430A20003102608840097
:100D40000008A1002508840003110318800A401040
:100D5000031940142108800740180314A503A603B3
:100D6000A20B9E2E08000230A2000314BA2E0430FB
:100D7000A2000314260884000008A10025088400AE
:100D8000031CC42E4010C92E8008401003194014C3
:100D900080032108800240180310A503A603A20BBC
:100DA000BA2E0800FF30B500B600B700B800053015
:100DB000A300E626A30BD92EB501B601B701B801F1
:100DC0000530A300E626A30BE22E08006430A00045
:100DD000F930A1000000A10BEA2EA00BE82E0800BC
:100DE0000A30A000F930A1000000A10BF42EA00BE6
:100DF000F22E08007C30A00000000000000000007F
:080E00000000A00BFC2E08000D
:101000000F398A018A158207DB348234E934E334EC
:10101000B23473347B348334FB34F334BA347934EC
:101020005834B93420340034C301830108308A00B5
:1010300043080F3982072B283E285028B428C92896
:10104000002932295C297C299C29BC29DC29102A09
:10105000222A562A6D2A83017330B5007930B600F2
:101060007C30B700BD30B80041183928C118392884
:101070003D284110C1100130C3006F2A7730B50000
:101080009F30B6007C30B7006E30B80041184B2856
:10109000C1184B284F284110C1100230C3006F2ADD
:1010A0004B0803196F28AA00A901A8018A019925F4
:1010B00008308A00B108031D6428FF30B100B00871
:1010C000031D6428FF30B000B50131080020B600D0
:1010D00030080020B7002F080020B8007728203003
:1010E000B5002030B6002030B7002030B800411CD9
:1010F000AD2841104B08003C031D81280330CB0074
:10110000B3284B08033C031D88280A30CB00B328C2
:101110004B080A3C031D8F281E30CB00B3284B0818
:101120001E3C031D96283C30CB00B3284B083C3CAA
:10113000031D9D287830CB00B3284B08783C031D55
:10114000A428B430CB00B3284B08B43C031DAB2813
:10115000F030CB00B328CB01B328C11CB328C11099
:10116000A9220330C3006F2AEA30B5008230B600EE
:101170007730B7009F30B8004118C128C118C12886
:10118000C8284110C1100430C300530E0339A30016
:101190006F2A2308031DD528FB30B500FB30B600AD
:1011A000FF30B700FB30B800F0282308013C031DD6
:1011B000E228FF30B500FB30B600FB30B700FB3053
:1011C000B800F0282308023C031DEF28FB30B500CF
:1011D000FF30B600FB30B700FB30B800F028A301A9
:1011E000411CF7284110230A0339A300FF28C11C22
:1011F000FF28C110230ED300A3220530C3006F2A9D
:1012000083013D30B500DB30B6003930B7007730B0
:10121000B80041180E29C1180E2931294110C110FA
:101220005008A8005108A9005208AA00C010A81F21
:101230002B29C014AC01AD01AE012E30A5002A301F
:10124000A6008A01B72608308A002C08A8002D08BD
:10125000A9002E08AA008A01992508308A000630C4
:10126000C3006F2A8630B5000430B600C01C3B298D
:101270002030B7003D290430B70034080020B80002
:10128000411C4E294110340A0F39B4003408093C7E
:1012900003185B29B4010230C0065B29C11C5B291D
:1012A000C110D001D101D201A801A9013408AA00BE
:1012B000C3220730C3006F2AED30B5000430B600FA
:1012C0000430B70033080020B800411C71294110D8
:1012D000330A0F39B3003308093C03187B29B301E3
:1012E0007B29C11C7B29C110A801A9013308AA00D0
:1012F000C3220830C3006F2AE730B5000430B600BF
:101300000430B70032080020B800411C9129411078
:10131000320A0F39B2003208093C03189B29B20186
:101320009B29C11C9B29C110A801A9013208AA0050
:10133000C3220930C3006F2AB630B5000430B600AE
:101340000430B70031080020B800411CB129411019
:10135000310A0F39B1003108093C0318BB29B1012A
:10136000BB29C11CBB29C110A801A9013108AA00D1
:10137000C3220A30C3006F2A7730B5000430B600AC
:101380000430B70030080020B800411CD1294110BA
:10139000300A0F39B0003008093C0318DB29B001CE
:1013A000DB29C11CDB29C110A801A9013008AA0052
:1013B000C3220B30C3006F2A7F30B5000430B60063
:1013C0000430B7002F080020B800411CF12941105B
:1013D0002F0A0F39AF002F08093C03180F2AAF015D
:1013E0000F2AC11C0F2AC110A801A9012F08AA00A9
:1013F000C322C01C0C2AAA01A901A8012A30A500F9
:101400005230A6008A01B72608308A002A08D20086
:101410002908D1002808D0008F220C30C3006F2A81
:10142000BB30B5002E30B6008230B7002E30B80089
:1014300041181D2AC1181D2A212A4110C1100D3042
:10144000C3006F2AB5014A080339CA00031D2F2AB9
:10145000DF30B600E930B7007330B800482A4A08D8
:10146000013C031D392AB601DF30B7007330B800E4
:10147000482A4A08023C031D432AB6018630B700B9
:10148000DB30B800482AB601ED30B700DB30B800D9
:10149000411C4F2A41104A0A0339CA00552AC11C6F
:1014A000552AC1109D220E30C3006F2AEA30B500C4
:1014B000DB30B6002A30B7007930B800411C642A0E
:1014C00041100130C3006C2AC11C6C2A4B08CC00AF
:1014D0005308C3008A0187286F2A8A013E2887198A
:1014E0007E2A42080311473C031DC20A4208031129
:1014F000463C0319C1140319C1178A2A4208031470
:10150000023C0318882AC11B882A4114C1178A2A61
:10151000C201C1138A01F02608308A001528830110
:101520000030A5005008AF220130A5005108AF22BD
:101530000230A5005208AF22080083010330A50045
:101540004A08AF22080083010430A5005308AF22E7
:10155000080083010530A5004B08AF220800830175
:1015600003178C008301250803178D0083168C0157
:101570000C1555308D00AA308D008C148C18BE2AA5
:101580000C118301080083010310D20DD10DD00D81
:101590002A30A5005230A6008A019B2608308A0016
:1015A0000310D20DD10DD00D0310D20DD10DD00DE1
:1015B0005230A5002A30A6008A019B2608308A00F6
:0215C000080021
:00000001FF
